:100000000C9475000C9492000C9492000C94920045
:100010000C9492000C9492000C9492000C94200189
:100020000C9492000C9492000C9492000C94841105
:100030000C9421110C9492000C9492000C94920058
:100040000C9492000C9492000C944B130C9492001C
:100050000C9423130C9492000C9492000C94920034
:100060000C9492000C94920039014501F9015C0155
:10007000680174018F01CB01B801DC01EA01A10D17
:10008000BD0DBD0DBD0DBD0DBD0DBD0DBD0DBD0D20
:10009000A90A710ABD0DBD0DBD0DBD0DBD0DBD0D76
:1000A000BD0DBD0DBD0D460D110C6A0D750D940DE8
:1000B000BD0DBD0D7009BD0D7B0D880DC90A8E0DDE
:1000C000BD0D000DAD0CDF0C9509FE09DB09210A01
:1000D000440A9209600A660AF90C54099E11AD118E
:1000E000BE11CB11DC11E911FC1111241FBECFEFA1
:1000F000D8E0DEBFCDBF11E0A0E0B1E0E0EBF9E277
:1001000002C005900D92A234B107D9F724E0A2E411
:10011000B1E001C01D92AA34B207E1F70E942006A7
:100120000C94D6140C940000A2E4B1E0E0E090E05E
:1001300021E02E0FE81721F03D919327E22FF8CF11
:10014000F0E0EE5BFE4F9083209349010895482F25
:1001500089E0E2E4F1E0DF011D928A95E9F7209160
:100160004D0130910101222351F0206C2093420176
:100170003093430182E0E42FF92F680F04C03093DD
:10018000420181E0F8CF861741F09191A82FB0E0AD
:10019000AE5BBE4F9C938F5FF6CF0E94940082E4CB
:1001A00091E008951092B00082E08093B10088E061
:1001B00080934E0110924C0110924B010895CF9301
:1001C000DF93EC0180915C0181112EC08F81823020
:1001D00068F18881882351F189E0FE01A3E5B1E04F
:1001E00001900D928A95E1F710925D0181E0809374
:1001F0005C018F81815080935B018CE08093520180
:10020000109250011092B20088E68093B30095B12D
:1002100080914E018095892385B98091700082601C
:100220008093700081E003C080E001C08FEFDF9118
:10023000CF91089581E090915C01911180E0089543
:100240001F920F920FB60F9211242F938F939F93AB
:10025000AF93BF93EF93FF93E0915D018E2F90E0FA
:100260008B30910508F0C5C0FC01EC5CFF4F0C948D
:10027000661495B180914E01892B85B98091B200A9
:1002800088598093B30081E0A2C095B180914E015E
:100290008095892385B98091B20088598093B300F5
:1002A00080915201815080935201882319F010925D
:1002B0005D019FC083E08BC095B180914E01892B79
:1002C00085B98091B20088528093B30084E07FC0EA
:1002D00095B180914E018095892385B98091B200B6
:1002E00088528093B30063C095B180914E01892BF1
:1002F00085B9E0915001F0E0ED5AFE4F2081209346
:100300004F018091B20090915101922311F498ED28
:1003100001C098E6890F8093B30086E058C095B17C
:1003200080914E018095892385B98091B2002091FA
:100330004F0190915101922311F498ED01C098E67C
:10034000890F8093B300809151018695809351016C
:10035000811130C0809150018F5F80935001909146
:100360005B019817B0F080E88093510187E02FC0BF
:1003700095B180914E018095892385B98091B20015
:1003800088528093B3009091500180915B0189174E
:1003900070F489E01CC095B180914E01892B85B91C
:1003A0008091B20088528093B30088E010C080E84A
:1003B0008093510185E00BC095B180914E01892B4E
:1003C00085B98091B20088598093B3008AE0809308
:1003D0005D010FC095B180914E018095892385B94B
:1003E0001092B200809170008D7F80937000109207
:1003F0005C01FF91EF91BF91AF919F918F912F91F0
:100400000F900FBE0F901F901895809300010895D4
:10041000809100010895E2E4F1E08FE7808311828A
:1004200082E00E94940082E491E00895CF93DF93EC
:1004300000D0CDB7DEB79FE3998390910001892B5F
:100440008A8362E0CE0101960E94A7000F900F9070
:10045000DF91CF910895CF93DF9300D01F92CDB756
:10046000DEB79CEE998381508A836B8363E0CE0173
:1004700001960E94A7000F900F900F90DF91CF91EF
:100480000895CF93DF931F92CDB7DEB78F71806849
:10049000898361E0CE0101960E94A7000F90DF9151
:1004A000CF910895CF93DF931F92CDB7DEB78F70B2
:1004B000806B898361E0CE0101960E94A7000F90B6
:1004C000DF91CF910895CF93DF931F92CDB7DEB721
:1004D0008F70806A898361E0CE0101960E94A70037
:1004E0000F90DF91CF910895CF93DF9300D0CDB7D8
:1004F000DEB79EED99838A8362E0CE0101960E9469
:10050000A7000F900F90DF91CF910895CF93DF93C5
:1005100000D0CDB7DEB79FED99838A8362E0CE012C
:1005200001960E94A7000F900F90DF91CF91089540
:1005300081E090E00C94A514BC0181E090E00C9463
:10054000C11480E090E00C949714682F80E090E054
:100550000C94AB1483E090E00C949714682F83E024
:1005600090E00C94AB1484E090E00C949714682F06
:1005700084E090E00C94AB148EE090E00C949F1417
:10058000AB01BC018EE090E00C94B9148AE090E0DD
:100590000C949F14AB01BC018AE090E00C94B91458
:1005A00086E090E00C949F14AB01BC0186E090E0E3
:1005B0000C94B91485E090E00C949714682F85E0B2
:1005C00090E00C94AB1485E190E00C949714682FA4
:1005D00085E190E00C94AB1484E190E00C949714C6
:1005E000682F84E190E00C94AB1483E190E00C94CC
:1005F0009714682F83E190E00C94AB1482E190E0B3
:100600000C949714682F82E190E00C94AB1486E16F
:1006100090E00C94A514BC0186E190E00C94C11408
:1006200083E390E00C949714682F83E390E00C949C
:10063000AB1490E0865D9F4F0C94971490E0865D1C
:100640009F4F0C94AB1490E08F5D9F4F0C949714C8
:1006500090E08F5D9F4F0C94AB1490E0885E9F4FAD
:100660000C94971490E0885E9F4F0C94AB1486E333
:1006700090E00C949714682F86E390E00C94AB14F0
:1006800085E390E00C949714682F85E390E00C9438
:10069000AB1484E390E00C949714682F84E390E00B
:1006A0000C94AB1487E390E00C949714682F87E3C5
:1006B00090E00C94AB1489E390E00C949714682FAD
:1006C00089E390E00C94AB1488E390E00C949714C9
:1006D000682F88E390E00C94AB148DE390E00C94C9
:1006E000A514BC018DE390E00C94C1148BE390E061
:1006F0000C94A514BC018BE390E00C94C1148AE324
:1007000090E00C949714682F8AE390E00C94AB145B
:1007100081E590E00C949714682F81E590E00C94AB
:10072000AB1487E490E00C94A51483E490E00C945F
:10073000A5148FE390E00C94A51489E490E00C9448
:10074000A51485E490E00C94A51481E490E00C9449
:10075000A514BC0187E490E00C94C114BC0183E4AF
:1007600090E00C94C114BC018FE390E00C94C11490
:10077000BC0189E490E00C94C114BC0185E490E0D4
:100780000C94C114BC0181E490E00C94C11485E583
:1007900090E00C94A514BC0185E590E00C94C11484
:1007A00084E590E00C949714682F84E590E00C9415
:1007B000AB144F706F70282F2F7034E6439FC00129
:1007C0001124820F911D2AE0629F800D911D11243A
:1007D0000895CF93C22F0E94D903CF7048EE53E003
:1007E000C49F9001C59F300D1124820F931FCF919C
:1007F00008958091840181110EC08091B60281110B
:1008000002C05E9A01C05E9880913504811102C0D9
:100810005D9A08955D98089580919C0199E0989F54
:10082000F0011124E951FD4FA9EAB2E001900D92C7
:100830009A95E1F78F5F803218F480939C0102C093
:1008400010929C0189EA92E00895FC0190919B012D
:1008500029E0299FD0011124A951BD4F01900D928B
:100860002A95E1F79F5F903218F490939B010895C9
:1008700010929B010895882349F0FA01862F09956B
:1008800090938202809381020C94250408957F92B4
:100890008F929F92AF92BF92CF92DF92EF92FF9290
:1008A0000F931F93CF93DF93C9E2D1E086E3882EA5
:1008B00084E0982E95E2E92E94E0F92E0CE014E005
:1008C000712C6881F40161934F0157018981F7010F
:1008D00081937F0168018A81F80181938F01872DBF
:1008E0000E943203F5016081872D0E941E03F601EC
:1008F0006081872D0E94280373942396F8E07F126D
:10090000E0CFDF91CF911F910F91FF90EF90DF909B
:10091000CF90BF90AF909F908F907F9008956091FF
:10092000890270918A0280E00E94331260911F0454
:100930007091200481E00E94331260912104709133
:10094000220482E00C9433120E94910390938A0255
:10095000809389020E9478120E949503909320044C
:1009600080931F040E9481120E9499039093220495
:10097000809321040C948A120E949D039093880214
:10098000809387020E9493120E94A1039093E50234
:100990008093E4020E949C120E94A50390931C0481
:1009A00080931B040C94A51282E00E94560380E001
:1009B00090E00E94CB0380E00E94D40380E00E947C
:1009C0008C0380E090E00E94A90380E090E00E9408
:1009D000AE0380E090E00E94B30388EE93E00E94B3
:1009E000B80388EE93E00E94BD0388EE93E00E9476
:1009F000C20380E00E943B0380E10E94440380E147
:100A00000E944D0383E090E00E94710380E090E03B
:100A10000E947A0380E00E94830380E00E946803C2
:100A200080E30E945F0384E00E94E70285E00E9469
:100A3000F00280E00E94F90280E00E9402030E941E
:100A4000470481E090E00E940B0380E00E941403C1
:100A500084E10E94D40268E270E080E090E00E94AD
:100A6000C0026EE170E080E090E00E94CA028BE07C
:100A70000E94DE0280E00E94AE0283E090E00E94CD
:100A80009C0280E00C94A5028D31A8F4982F9695D5
:100A900096959695ECE0E91BF0E0E557FD4F208137
:100AA00030E08770A90102C0559547958A95E2F715
:100AB000CA018170089580E00895809171018823B2
:100AC00071F090916F0180917001209197029223B3
:100AD0009093970290919602892380939602209199
:100AE0009702622F66956F70922F91709295907F0A
:100AF000692B6093340490919602892F8170880F3E
:100B0000880F880F322F329536953770832B80935C
:100B10006201892F86958F708093610130919502D3
:100B200088E0389FA0011124929596959770942B98
:100B3000909360019091940248E0949FC001112429
:100B4000329536953770832B80935F0120935E0139
:100B5000809166018227809366018F7121F041E4C4
:100B600052E00E943B0480916601807E31F042E5B4
:100B700052E0609162010E943B0480915E0180938B
:100B800066019091960290935E018091650189279C
:100B90008093650180FF07C042E552E060916201E9
:100BA00081E00E943B04809165018E7131F043E643
:100BB00052E0609161010E943B0480916501807E5A
:100BC00031F044E752E0609160010E943B04809163
:100BD0005E01809365019091950290935E018091F2
:100BE00064018927809364018F7131F044E752E0FA
:100BF000609160010E943B0480916401807E31F02D
:100C000046E852E060915F010E943B0480915E01E2
:100C1000809364019091940290935E0180916301AE
:100C20008927809363018F7131F046E852E060912B
:100C30005F010E943B0480915E01809363010895EF
:100C40008FE384B987B1886C87B988B18F6388B91D
:100C50000E94F7100E94D20080EE8AB985B1806EA2
:100C600085B90E94B302882329F00E94D40480E051
:100C70000E94B70286B1807280934204803211F0E4
:100C80000E94D4040E94C70390930A018093090133
:100C90000E94D0038093B702109268010E9437032C
:100CA000809315040E94400380939F020E94490391
:100CB000809340040E94880380933F040E94AE12F8
:100CC0000E94A4040E94BC040E948F0425E2C22E4C
:100CD00024E0D22E06E314E03CE0E32E34E0F32ED1
:100CE000C0E08C2F0E941903F60181936F018C2FB5
:100CF0000E942303F70181937F018C2F0E942D0313
:100D0000F80181938F01CF5FC83059F70E9410031B
:100D1000809371010E946D039093060180930501F9
:100D20000E9464038053809307010E945B038093B9
:100D300008010E947F03809398010E94760390939C
:100D40009A01809399010E945203809324040E9487
:100D500007039093700180936F010E94E3028093D8
:100D60000B040E94EC02809341040E94F5028093E0
:100D7000B6020E94FE02809335040E94D00290E0E9
:100D8000A0E0B0E08093880190938901A0938A014C
:100D9000B0938B010E94BC0260939001709391010B
:100DA00080939201909393010E94C60260938C01FC
:100DB00070938D0180938E0190938F010E94DA02CF
:100DC000809302010E94980290933304809332042E
:100DD0000E94A102809323040E94AA0280938401AE
:100DE00081110E94EB100E94F90380912404882352
:100DF00089F082508230E0F464EF71E080E00E947C
:100E0000331284EF91E090938601809385011092D4
:100E100095010EC06091890270918A0280E00E9463
:100E2000331260911F047091200481E00E943312FC
:100E300060E076E980E090E00E94B9120E94EA1238
:100E400078940E940B02909382028093810229E0A1
:100E5000FC01A8E7B2E001900D922A95E1F70E940B
:100E6000250480E00E941602909382028093810202
:100E700029E0FC01AFE6B2E001900D922A95E1F77E
:100E80000E9425048091090190910A010E94251277
:100E90000E942A1260939A0270939B0280939C0294
:100EA00090939D020E94F21290931704809316046F
:100EB000A8E26A2E08EE13E0B4EFCB2EDD24D39423
:100EC000CAE94C2EC2E05C2ED9EBED2ED2E0FD2E0D
:100ED0008EE1782E22242394312C80916901813077
:100EE000C9F120F08E3009F4C1C149C60E94FB123D
:100EF000803109F044C6A0911604B0911704EBE8C4
:100F0000F2E08D9181934E165F06D9F70E94F5129B
:100F1000809318040E9401130E94FE1290918B028C
:100F200080910701981312C090918C028091080162
:100F300098130CC080918D028F3041F48091900203
:100F4000833521F481E08093690119C6FEE0F093B6
:100F5000690115C6109269018091910290919202E7
:100F60009827892798272091910227FF03C0809115
:100F7000920290E0909304018093030120919302E8
:100F80002093960130919801809103019091040182
:100F9000332351F0323019F42058209396012091D8
:100FA000990130919A0104C0209105013091060108
:100FB0002817390729F08091970180939601DFC5A2
:100FC0008091960180780E940502809168018823B3
:100FD00021F1209193022F778091970190919601B2
:100FE000222369F0907890939601807880939701FE
:100FF000D0928601C0928501109295010EC0109288
:101000006801907890939601807880939701109270
:101010009501D0928601C092850110920B018091BA
:101020006801811106C08091090190910A010E9416
:10103000251280912404813009F441C058F0823097
:1010400009F465C0833009F08FC0809196018093C8
:1010500095018AC08091960187FF05C06091E402E6
:101060007091E50204C060911F047091200481E03A
:101070000E943312809196018F77809396012AE027
:10108000829FC0011124893E33E093072CF4909392
:101090001E0480931D0404C010931E0400931D04BD
:1010A00080911D0490911E0497FF04C010921E04AD
:1010B00010921D0460911D0470911E0453C0809114
:1010C000960187FF13C0809140040E944405882345
:1010D00041F060911B0470911C0482E00E94331265
:1010E00043C06091210470912204F7CF80919F0248
:1010F0000E944405882329F06091E4027091E50282
:1011000004C060911F047091200481E0E7CF0E9429
:101110000802909196019F77882329F0892F90E00B
:1011200083589F4F05C04DE750E0491B5109CA0144
:10113000880F991F880F991F90931E0480931D0498
:1011400060911D0470911E0477FF02C060E070E0A2
:10115000693E53E0750714F068EE73E070931E0467
:1011600060931D0480E0BACF20919601322F3F7723
:101170003093940180917101882321F1809168015D
:10118000811120C0ECE0F4E0A6E3B4E080E090E060
:101190004D91431790F04081341778F02078FC018E
:1011A000EB5DFB4F8081282B2093960180912404D6
:1011B000833041F42093950105C001963196883023
:1011C000910531F7809196018F770E9416029093D6
:1011D0008202809381020E9425048091960180936F
:1011E000970180918401811114C0C091B602809151
:1011F0000B040E944405C81302C05E9A01C05E98A9
:10120000C0913504809141040E944405C81307C071
:1012100004C00E940802882311F05D9A01C05D9805
:10122000809124048330F9F4809102010E944405E6
:1012300090918701882351F080916801811106C047
:101240009F5F993234F06092870108C0915097FDFA
:1012500003C09093870102C010928701809187019B
:101260008111109295010E945D0589C41092690157
:101270000E94F812EC0190938402809383022C81E7
:101280002093A6023D8130931A04E885E09367011C
:101290008E2F90E0FC017097EF32F10508F06DC4DD
:1012A000E15CFF4F0C9466142C854B856A8589851B
:1012B0000E94E903AC0160E070E040934604509363
:1012C000470460934804709349040E949C02E09193
:1012D0008302F091840281858F700E94A5024DC423
:1012E000F701272D11922A95E9F785E28093B9023B
:1012F00085E48093BA020E94A1028093BB020E94FF
:101300009802AC0160E070E04093460450934704BB
:1013100060934804709349048093BC02882790939B
:10132000BD0240C00E94D40428C4F701272D1192A9
:101330002A95E9F785E28093B90280E58093BA02A5
:101340000E94D002482F50E060E070E040934604D5
:101350005093470460934804709349048093BB0200
:101360001092BC020E94BC02609346047093470432
:1013700080934804909349046093BD027093BE0229
:101380000E94C60260934604709347048093480409
:10139000909349046093BF027093C0020E94DA02E6
:1013A0008093C10249EB52E060911A048091A60239
:1013B0000E94F013E2C34B856A8589850E94D90398
:1013C000BC0180E090E060934604709347048093F2
:1013D0004804909349040E94CA0280914604909167
:1013E0004704A0914804B091490480938C019093E4
:1013F0008D01A0938E01B0938F01BFC34B856A8589
:1014000089850E94D903BC0180E090E06093460486
:101410007093470480934804909349040E94C0024B
:101420008091460490914704A0914804B0914904EA
:101430008093900190939101A0939201B0939301B6
:101440009CC34B856A8589850E94D903AC0160E005
:1014500070E04093460450934704609348047093AF
:1014600049040E94D4028091460490914704A091BF
:101470004804B09149048093880190938901A09316
:101480008A01B0938B0179C38A858F7029852F706B
:101490003AE0839FC0011124820F911DAC0160E0EE
:1014A00070E040934604509347046093480470935F
:1014B00049040E94DE0280914604809302015DC3CC
:1014C0008985809384010E94AE0257C385E2809390
:1014D000B90287E58093BA02809184018093BB02B0
:1014E00037C2298530E03093A2012093A1018A857B
:1014F000482F50E05093A00140939F014B8550E04E
:1015000050939E0140939D012130310589F40E9442
:10151000E70280919F0180930B0480919D0181706F
:101520000E94F90280919D0181708093B60225C3CB
:101530000E94F00280919F018093410480919D015F
:1015400081700E94020380919D0181708093350417
:1015500014C3298530E03093A2012093A10181E0DA
:10156000232B09F480E08093B7020E94D4032091DA
:10157000A1013091A201209FC001219F900D309FB9
:10158000900D112490930A01809309010E94CB03CE
:10159000F4C289858F708093B8022A854B856C854B
:1015A0008D850E94E9039093A1028093A0022E856D
:1015B0004F85688989890E94E9039093E2028093AC
:1015C000E1028A89817080934304109244049B89CC
:1015D0009F708C898F704AE0949F800D11248093B6
:1015E0009E020E948803982F977090933F04209149
:1015F000B802213009F45DC020F0223009F4B1C0F6
:1016000007C12091430430914404232B21F48670B8
:1016100080933F0403C0916090933F040E94910324
:101620009C0190938A02809389028091E1029091BB
:10163000E2022817390799F090938A028093890271
:101640000E94A9038091E1029091E2020E94781227
:101650006091E1027091E20280E00E9433120E94E8
:101660009D039C0190938802809387028091A00241
:101670009091A1022817390799F0909388028093DE
:1016800087020E94B8038091A0029091A1020E945B
:1016900093126091A0027091A10280E00E94331227
:1016A00080919E020E943B0380919E0280931504CC
:1016B000AFC02091430430914404232B21F4857062
:1016C00080933F0403C0926090933F040E9495036F
:1016D0009C019093200480931F048091E1029091DB
:1016E000E2022817390799F09093200480931F0491
:1016F0000E94AE038091E1029091E2020E94811269
:101700006091E1027091E20281E00E9433120E9436
:10171000A1039C019093E5028093E4028091A002D2
:101720009091A1022817390799F09093E5028093D0
:10173000E4020E94BD038091A0029091A1020E9448
:101740009C126091A0027091A10281E00E9433126C
:1017500080919E020E94440380919E0280939F028A
:1017600057C02091430430914404232B21F483700B
:1017700080933F0403C0946090933F040E949903B8
:101780009C0190932204809321048091E102909126
:10179000E2022817390799F09093220480932104DC
:1017A0000E94B3038091E1029091E2020E948A12AA
:1017B0006091E1027091E20282E00E9433120E9485
:1017C000A5039C0190931C0480931B048091A002AC
:1017D0009091A1022817390799F090931C048093E7
:1017E0001B040E94C2038091A0029091A1020E945A
:1017F000A5126091A0027091A10282E00E943312B2
:1018000080919E020E944D0380919E02809340042D
:1018100080913F040E948C0380913F040E94AE128D
:10182000ACC182E2F70111928A95E9F785E28093D3
:10183000B90287E58093BA0280910701805D8093A9
:10184000BB02809108018093BC02909105018091B8
:1018500006019093BD028093BE0290919901809100
:101860009A019093BF028093C00280919801809367
:10187000C1029091890280918A029093C202809362
:10188000C30290918702809188029093C402809352
:10189000C50290911F04809120049093C60280930A
:1018A000C7029091E4028091E5029093C802809370
:1018B000C90290912104809122049093CA028093DE
:1018C000CB0290911B0480911C049093CC028093D6
:1018D000CD02809115048093CE0280919F02809367
:1018E000CF02809140048093D00280913F04809386
:1018F000D102809124048093D202809109019091B9
:101900000A01B8010E9433146093D3028091B60299
:10191000F0E88F9FC001112490910B04892B8093D4
:10192000D4028091350440E8849FC0011124909135
:101930004104892B8093D502909132048091330425
:101940009093D6028093D702809123048093D8028B
:1019500049EB52E0632F822F2BCD89858F708093C6
:101960006E019A85917090936D01F10102C0EE0FA6
:10197000FF1F8A95E2F7F0936C01E0936B010E94E0
:10198000070340916D0120916B0130916C0144235C
:1019900039F0822B932B9093700180936F0108C0D4
:1019A00020953095282339233093700120936F01BF
:1019B00080916F01909170010E940B03DEC0F701CE
:1019C000272D11922A95E9F734E33093B9028DE47B
:1019D0008093BA020E94070380936F019093700175
:1019E0008093BB029093BC020E9410038093BD02BF
:1019F000D9CC89858170809371010E941403BDC088
:101A000089858170809371010E941403E0918302A3
:101A1000F0918402C285CF70C150C093720143859A
:101A2000648585850E94D903EC2FF0E0EB5DFB4FC8
:101A30008083682F8C2F0E941E03C0917201E09159
:101A40008302F09184024685678580890E94D903CC
:101A5000EC2FF0E0E45FFB4F8083682F8C2F0E9417
:101A60002803C0917201E0918302F09184024189C0
:101A7000628983890E94D903EC2FF0E0EA5CFB4F76
:101A80008083682F8C2F0E94320377C0F701272DA7
:101A900011922A95E9F734E23093B9024EE440936B
:101AA000BA020E9410038093BB02C9EBD2E0912CD2
:101AB000892D0E9423038B83892D0E942D038C8303
:101AC000892D0E9419038D839394239658E09512D3
:101AD000EFCF68CC8985809307010E9468038091CD
:101AE000070180538093070148C0898580930801CE
:101AF0000E945F0342C029854A856B858C850E94C0
:101B0000E90390939A01809399010E947A0335C06A
:101B10008985809398010E9483032FC089858093D3
:101B200024040E94560329C029854A856B858C852B
:101B30000E94E90390930601809305010E947103BE
:101B40001CC029854A856B858C850E94E9034C0160
:101B50009093A3028093A2024E856F8588890E948C
:101B6000D90380931904682FC4010E942B0290931B
:101B70008202809381020E9425040E94FE128091BD
:101B80002404833009F064C10E942A1280909A02D2
:101B900090909B02A0909C02B0909D02DC01CB0132
:101BA00088199909AA09BB0980930704909308042E
:101BB000A0930904B0930A040E940802609187016F
:101BC000909195012091850130918601882309F437
:101BD00091C09F77892F90E083589F4F880F991F5E
:101BE000880F991F893EE3E09E072CF490931E0412
:101BF00080931D0404C010931E0400931D04809163
:101C00001D0490911E04843F914024F4D0921E0440
:101C1000C0921D046623E9F180916801811139C0E9
:101C20008090070490900804A0900904B0900A04E2
:101C30008091880190918901A0918A01B0918B01D6
:101C400088159905AA05BB0524F5261B310967FDF2
:101C50003395309386012093850180911D049091E6
:101C60001E042817390720F490938601809385017C
:101C7000609185017091860180E00E9433120E947C
:101C80002A1260939A0270939B0280939C02909315
:101C90009D0220911D0430911E0480918501909138
:101CA0008601821793078CF48090070490900804B3
:101CB000A0900904B0900A044091900150919101C4
:101CC0006091920170919301A0C0281739070CF020
:101CD000BFC08090070490900804A0900904B090C1
:101CE0000A0440918C0150918D0160918E01709198
:101CF0008F016EC04DE750E0491B5109CA01440FE6
:101D0000551F440F551F95FD05C050931E04409369
:101D10001D0404C010921E0410921D046623E9F1F4
:101D200080916801811139C0809007049090080467
:101D3000A0900904B0900A048091880190918901D3
:101D4000A0918A01B0918B0188159905AA05BB0560
:101D500024F5260F311D67FD3A95309386012093B7
:101D6000850180911D0490911E048217930720F431
:101D70009093860180938501609185017091860121
:101D800080E00E9433120E942A1260939A0270939C
:101D90009B0280939C0290939D0220911D043091A0
:101DA0001E04809185019091860128173907D4F48B
:101DB0008090070490900804A0900904B0900A0451
:101DC0004091900150919101609192017091930125
:101DD000481559056A057B05DCF5019782179307BD
:101DE00010F11CC0821793079CF580900704909017
:101DF0000804A0900904B0900A0440918C0150910D
:101E00008D0160918E0170918F01481559056A0509
:101E10007B05F4F401962817390728F09093860182
:101E20008093850104C030938601209385016091E1
:101E300085017091860180E00E9433120E942A126F
:101E400060939A0270939B0280939C0290939D02F0
:101E500080916801882309F445C00E94161264E647
:101E600070E00E943314EB010E940802882361F0A5
:101E7000CE0183589F4F880F991F880F991F893E65
:101E800053E095076CF41BC08DE790E08C1B9D0B15
:101E9000880F991F880F991F893EE3E09E077CF009
:101EA00010931E0400931D0480911D0490911E0444
:101EB00097FF0AC010921E0410921D0405C0909353
:101EC0001E0480931D04F0CF60911D0470911E04C8
:101ED00080E00E943312C13019F0C093960102C015
:101EE000109296018091B7028823E1F10E9420129E
:101EF00018161906BCF180912404833039F58091BD
:101F00006801811123C00E9408022091850130914F
:101F10008601882321F0C901845F914003C0C60176
:101F2000821B930B97FD03969595879595958795BD
:101F30008F77992724E6AC01249FC001259F900D3F
:101F400011240E941B1281E0809368018091240477
:101F5000811106C06091A4027091A5020E94331203
:101F60000E94F90380918401882309F4EFC0C09195
:101F70009601C0939501809102010E944405209131
:101F8000680190918301882341F0211106C09F5F71
:101F9000993234F06092830108C0915097FD03C0DC
:101FA0009093830102C0109283018091830181117B
:101FB000109295012111C7C00E942A1280902E0410
:101FC00090902F04A0903004B0903104AB01BC017C
:101FD000481959096A097B094093B2025093B30228
:101FE0006093B4027093B502809195018F7790E071
:101FF0009093740180937301E0918301EE2379F152
:102000002091680121112BC0809077019090780178
:10201000A0907901B0907A0184169506A606B706BD
:10202000F4F420917501309176012E1B3109E7FD02
:1020300033952817390728F03093760120937501DE
:1020400004C090937601809375010E942A126093D8
:102050002E0470932F0480933004909331042091C8
:10206000730130917401E0917501F0917601E217EE
:10207000F3076CF58091B2029091B302A091B40283
:10208000B091B50240917F01509180016091810132
:1020900070918201481759076A077B07C4F4CF0182
:1020A00001962817390728F09093760180937501DF
:1020B00004C030937601209375010E942A12609328
:1020C0002E0470932F048093300490933104209158
:1020D000730130917401E0917501F09176012E1732
:1020E0003F076CF58091B2029091B302A091B402C7
:1020F000B091B50240917B0150917C0160917D01CE
:1021000070917E01481759076A077B07C4F4CF0115
:1021100001978217930728F09093760180937501B9
:1021200004C030937601209375010E942A126093B7
:102130002E0470932F048093300490933104809187
:102140007501880F01C08C2F0E94F51080916A01E3
:102150008A3088F40E941A01882311F40C946D07C8
:102160008FE692E00E94DF0080916A018F5F80938A
:102170006A010C946D0790919C0180919B019817C6
:1021800069F00E940C0429E0FC01AFE6B2E0019086
:102190000D922A95E1F710926A0111C08091960183
:1021A0008F770E941602909382028093810229E029
:1021B000FC01AFE6B2E001900D922A95E1F70E9492
:1021C0001A01882311F40C946D078FE692E00E94A7
:1021D000DF000C946D07569A8FEB87BD84B583683A
:1021E00084BD85B5826085BD089587BD0895109230
:1021F000A3011092A4011092A5011092A6018FE3F1
:1022000084B91092A90110928000E1E8F0E01082F8
:10221000109285001092840080E09DE790938900E1
:102220008093880080ED97E090938B0080938A00E4
:10223000808182608083EFE6F0E080818660808329
:1022400008951F920F920FB60F9211248F939F93B0
:10225000AF93BF9380910C0190910D011816190650
:102260009CF480910C0190910D01019790930D01C8
:1022700080930C0180910C0190910D0197FF04C097
:1022800010920D0110920C018091A7019091A8016C
:10229000181619069CF48091A7019091A801029745
:1022A0009093A8018093A7018091A7019091A80124
:1022B00097FF04C01092A8011092A7018091A3017A
:1022C0009091A401A091A501B091A6010196A11D34
:1022D000B11D8093A3019093A401A093A501B09395
:1022E000A60180918400909185008053984F90932F
:1022F0008B0080938A00BF91AF919F918F910F9037
:102300000FBE0F901F9018951F920F920FB60F924D
:1023100011242F933F938F939F93AF93BF93EF938A
:10232000FF93E091A9018E2F90E08730910508F08E
:1023300070C0FC01E259FF4F0C94661485B1887F90
:1023400085B980918800909189008053984F90932F
:1023500089008093880081E04CC0289A20910E016A
:1023600030910F018091880090918900820F931F16
:10237000909389008093880082E03BC028988091E8
:102380008800909189008053984F909389008093A2
:10239000880083E02EC0299A2091170130911801FE
:1023A0008091880090918900820F931F90938900FB
:1023B0008093880084E01DC02998809188009091C6
:1023C00089008053984F909389008093880085E01E
:1023D00010C02A9A2091200130912101809188001B
:1023E00090918900820F931F9093890080938800B9
:1023F00086E08093A9010DC02A9880918800909171
:102400008900805E914B90938900809388001092A0
:10241000A901FF91EF91BF91AF919F918F913F9152
:102420002F910F900FBE0F901F9018958091A701CC
:102430009091A80108959093A8018093A701089511
:1024400080910C0190910D01089590930D0180935E
:102450000C0108956091A3017091A4018091A501E0
:102460009091A6010895833008F041C0693E43E091
:102470007407E8F5282F30E059E0859FF00111241A
:10248000E25FFE4F828193816817790714F46281BD
:10249000738189E0829FF001839FF00D1124E25F38
:1024A000FE4F848195818617970714F464817581A6
:1024B00089E0829FF001839FF00D1124E25FFE4FBF
:1024C0008085882331F088EE93E0AC01461B570BE2
:1024D000BA0168517C4F660F771F89E0829FF00137
:1024E000839FF00D1124E25FFE4F71836083089596
:1024F000893E23E0920720F490931101809310010C
:102500000895893E23E0920720F490931A01809366
:1025100019010895893E23E0920720F49093230146
:10252000809322010895893E23E0920720F490933E
:102530001301809312010895893E23E0920720F44D
:1025400090931C0180931B010895893E23E092071C
:1025500020F490932501809324010895982F917081
:10256000EEE0F1E09087982F9270918B8470828FCB
:1025700008959B01AC0184E0220F331F441F551FB7
:102580008A95D1F760E074E284EF90E00E944714EE
:10259000BA01A901415051096109710988E180938B
:1025A000C1008EE08093C2004093C400BB2777FD3A
:1025B000BA95A72F962F852F8093C5001092AA0158
:1025C0001092B10180E3EFE3F2E0DF011D928A9502
:1025D000E9F70895E1ECF0E0808180688083109253
:1025E000B101089587E192E0089580911202089563
:1025F0008FE092E008958091AD0108951092AD01B1
:1026000008958093B2010895CF93C1E0C093AE01C5
:102610006093AF01462F50E0BC018FED91E00E9426
:102620008E148091DF018093C600E1ECF0E08081A0
:1026300080648083E0ECF0E0808180648083C093DC
:10264000B001CF9108951F920F920FB60F921124EF
:102650008F93EF93FF93E091B0018091AF01E81762
:1026600040F08091C1008F7B8093C1001092AE0139
:102670000AC081E08E0F8093B001F0E0E152FE4F7E
:1026800080818093C600FF91EF918F910F900FBED4
:102690000F901F9018951F920F920FB60F92112452
:1026A0002F933F934F935F936F937F938F939F935A
:1026B000AF93BF93EF93FF938091C6009091AA01CF
:1026C000923059F1A8F49923C9F0913009F077C0FC
:1026D000E091B10191E09E0F9093B101F0E0E15CD7
:1026E000FD4F80831092AB018093AC0182E02CC03F
:1026F000933069F1963008F442C061C08E3709F01A
:102700005EC0E091B10191E09E0F9093B101F0E0C5
:10271000E15CFD4F808381E017C0E091B10191E061
:102720009E0F9093B101F0E0E15CFD4F808320911A
:10273000AB013091AC01A901482BCA0102969093DC
:10274000AC018093AB0183E08093AA0138C0E09193
:10275000B10191E09E0F9093B101F0E0E15CFD4F7B
:102760008083883829F08D3A29F0813829F402C015
:1027700084E0EACF85E0E8CF1092B1011EC0E0917D
:10278000B10191E09E0F9093B101F0E0E15CFD4F4B
:1027900080834091AB015091AC01892F90E04817A4
:1027A000590768F46FE372E08FE092E00E948E14A4
:1027B0001092B10180E18093AD011092AA01FF91C6
:1027C000EF91BF91AF919F918F917F916F915F91A9
:1027D0004F913F912F910F900FBE0F901F90189522
:1027E0009EE79093B3011092B40196E29093B501E5
:1027F00091E09093B6011092B7018093B801609375
:10280000B9011092BA0182E2FA01ABEBB1E001909A
:102810000D928A95E1F7E6EBF1E080E09191890F66
:1028200091E0EC3DF907D1F780958093DC016AE2F5
:1028300083EB91E00E94041383EB91E00895AA1BBF
:10284000BB1B51E107C0AA1FBB1FA617B70710F09B
:10285000A61BB70B881F991F5A95A9F780959095CD
:10286000BC01CD01089597FB072E16F4009407D004
:1028700077FD09D00E941F1407FC05D03EF4909507
:1028800081959F4F0895709561957F4F0895052E0E
:1028900097FB1EF400940E945E1457FD07D00E941F
:1028A0006C1407FC03D04EF40C945E1450954095C4
:1028B000309521953F4F4F4F5F4F089590958095EC
:1028C000709561957F4F8F4F9F4F0895EE0FFF1FBB
:1028D0000590F491E02D0994A1E21A2EAA1BBB1BCE
:1028E000FD010DC0AA1FBB1FEE1FFF1FA217B307DC
:1028F000E407F50720F0A21BB30BE40BF50B661FF2
:10290000771F881F991F1A9469F7609570958095B5
:1029100090959B01AC01BD01CF010895FB01DC0145
:1029200002C001900D9241505040D8F70895F99996
:10293000FECF92BD81BDF89A992780B50895A6E192
:10294000B0E044E050E00C94C814A8E1B0E042E0EC
:1029500050E00C94C814262FF999FECF1FBA92BDEF
:1029600081BD20BD0FB6F894FA9AF99A0FBE019670
:102970000895242F0E94AC14252F0E94AC140C94AF
:10298000C1140E94AB14272F0C94AC14DC01CB01B2
:10299000FC01F999FECF06C0F2BDE1BDF89A31966F
:1029A00000B40D9241505040B8F70895F894FFCF0D
:1029B00080030703000300D030B80B01B80BD00729
:1029C0000000D007D00700D0070000D007D00700D4
:1029D000D0070000D007D0070008070618171628F0
:1029E00027263837364847465857566867667877F7
:0229F00076006F
:00000001FF
